:1000000011298030A100FE30AF200130AF207530C3
:10001000A7003030C628A101A117AF00AF08031D0B
:100020001328030114280130AF020310A20CA20C04
:10003000A20CC0302205403EAF07FE30AF202F0893
:10004000AF28A101A117AF00FE30AF202F08AF28C5
:10005000A401AA00AB01A01124080319A0150530C2
:10006000A3002730A900103041200330A900E83058
:100070004120A90164304120A9010A3041202A0809
:100080004828A8002B08A7002A08A600DA2026087E
:10009000A600A3030319A011240803195228230260
:1000A000031859282608031DA011A0195928303E0D
:1000B000AF280800A300240803190C292308AF2047
:1000C000A4035B28AD000611861183160611861164
:1000D0000F30860583122D08A0188C283E30A7000B
:1000E0008030C6203330AC00A0201330A700883009
:1000F000C620A0206430C520A0206430C520223056
:10010000AC00A02028308B200C308B2006308B20B8
:10011000A0142D088C282014AC00201C9A288611CD
:10012000033C031C9F289F200530A700DC30C6201D
:10013000031408002014FE3C0319AD288615201C6A
:10014000201006150F3086052C08F039860406119C
:10015000AC0E2018A0283230C5202D080C29A11B78
:10016000622883178001840AFF3E031DB2280C29F0
:10017000A901A800FF30A807031CA907031C0C292C
:100180000330A700DF30C620BA28A701E83EA6004A
:10019000A709FC30031CCF28A6070318CC28A60704
:1001A0000000A70FCC282618D528A61CD9280000A7
:1001B000D9280800AB01AA011030AC00270DAA0D08
:1001C000AB0D2808AA022908031C290FAB0203184B
:1001D000F0282808AA0729080318290FAB070310DD
:1001E000A60DA70DAC0BDE2826080C291030B00098
:1001F000A701A601AD0CAC0C031C04292808A60716
:1002000029080318290FA707A70CA60CAB0CAA0CEA
:10021000B00BFA282A080C29831383120313000059
:100220000800A00107309F00E03083168500FF30F2
:10023000860081138312850186012030840060309E
:10024000B220A03084005030B22020308400303002
:10025000B120C830B82001207730622062206220AF
:100260002E3062207030622069306220633062205C
:100270006230622061306220733062206930622017
:10028000633062202E3062206E3062206C3062203B
:100290000B30A900B830B92001204430622043302F
:1002A0006220463062203130622036306220553084
:1002B00062204B3062204130622020306220622078
:1002C000563062202D306220323062200730A90083
:1002D000D030B920012041306220643062206A3081
:1002E00062207530622073306220743062202030CA
:1002F00062204C30622044306220523062208618E6
:100300008729851F85290514862905107F29012045
:10031000533062206530622061306220723062208A
:1003200063306220683062202030622073306220A7
:1003300069306220673062206E3062206130622056
:100340006C30622036140512831605128312282A97
:10035000C3013C03A500C90149082502031CC129AA
:10036000E421B61CBF294308A6004908A200A60143
:10037000A20A0314A60DA20BBA292608C304C90FAA
:10038000AC29B2014308B100B20CB10CB20CB10CF3
:10039000B20CB10CB20CB10C0F30B2053208AD008A
:1003A0003108AC00A9010A30A800F620B1002B08E2
:1003B000B200B4014308B3000F30B3050030B405F8
:1003C00031083307C3000800BA01B9010618F9293A
:1003D0000130B820B90A0319BA0A0B303A02031CDB
:1003E000F829031DF729B9303902031CF8295B2CC1
:1003F000E6299B30B8200618B614061CB610361C29
:10040000122A440EB100B200F030B1050F30B2052F
:100410003208A7003108A600A9013A30A800DA2066
:10042000BD001B2A03013619013EB618013A031913
:100430003611031D3615C40A85140130A900F430A5
:10044000B9208510A901F030A8002808B9200800BB
:10045000BB01C4013612361AB32ABA01B901061C0F
:10046000422AB90A0319BA0A0130B820AF303A0259
:10047000031C412A031D402AC9303902031C412AAA
:100480005B2C2F2ABA01B9010618742AB90A03197C
:10049000BA0A0A30B8203618682A39080B3A3A04E2
:1004A000031D532A672A3908193A3A04031D5A2AA8
:1004B0008514672A39084B3A3A04031D612A8510CE
:1004C000672A3908FA3A3A04031D672A5B2C732A13
:1004D00011303A02031C732A031D722A9530390227
:1004E000031C732A5B2C442A41303B02031C792AEB
:1004F0005B2CBB0A3A08031D812A65303902031CB4
:10050000822A3616361CB22A3B0EB100B200F030F9
:10051000B1050F30B2053208A7003108A600A901C5
:100520004130A800DA20BD008030A10080302120B9
:10053000463062206F306220753062206E3062205B
:100540006430622020306220733062206930622083
:10055000673062206E306220613062206C30622031
:10056000203062202B2A361CCF2A012049306220FD
:100570006E306220693062207430622069306220FF
:10058000613062206C306220693062207A306220F3
:10059000653062202E30622062206220342B0B30C6
:1005A000BD000130A2003D080B20A101B61DE72AC5
:1005B0003B3041020318DE2AC10AE62AC101173086
:1005C00045020318E52AC50AE62AC501EB2A4208B6
:1005D000C1004608C500051BFB2A4508031DF32A78
:1005E0000C30C700FA2A0D304502031CFA2A0C30E1
:1005F0004502C700FF2A4508C700203062200A30A4
:1006000047020318052B203062208030A1004708E4
:1006100028203A3062200230A40041082920051B1E
:100620001D2B0C3045020318182B613062201A2B49
:10063000703062200E30BD001F2B0F30BD0041080E
:1006400003190130031D0301B5001E3041020319D7
:100650000130031D03013504B50001308618030184
:1006600035040319342B332C361E312CE421013090
:10067000C9000F3049020318402BE421C90F392B60
:100680003611B611E421E421E421B61C492B0514EE
:100690004A2B05101230C900143049020318532B9D
:1006A000E421C90F4C2BE4210730BC00A8214308EA
:1006B000C200E421361D5D2BB6150630BC00A82112
:1006C0004308C600E421361D662BB6150630BC0073
:1006D000A8214308BE000330BC00A8214308C8007D
:1006E0000530BC00A8214308C0000830BC00A82188
:1006F0004308BF00E421361D7E2BB615361C842B23
:10070000B619832B36100120B619302C8030A10089
:10071000C03021201030A40020305A208030A100A9
:10072000803021203E082820203062200130400205
:10073000031DA12B4A306220613062206E3062209E
:10074000192C02304002031DAC2B4630622065306C
:10075000622062306220192C03304002031DB72B47
:100760004D3062206130622072306220192C0430DA
:100770004002031DC22B4130622070306220723073
:100780006220192C05304002031DCD2B4D30622014
:100790006130622079306220192C06304002031D3E
:1007A000D82B4A306220753062206E306220192CBE
:1007B00007304002031DE32B4A306220753062206F
:1007C0006C306220192C08304002031DEE2B4130A2
:1007D00062207530622067306220192C0930400297
:1007E000031DF92B53306220653062207030622087
:1007F000192C0A304002031D042C4F306220633054
:10080000622074306220192C0B304002031D0F2C23
:100810004E3062206F30622076306220192C0C300E
:100820004002031D192C4430622065306220633081
:100830006220051B262C203062208030A10002306F
:10084000A4003F08292020306220302C2030622074
:10085000273062208030A1000230A4003F08292008
:10086000322C5B2C282A851F3A2C05128316051280
:1008700083123C2C8316051683129B30B820410846
:1008800003190130031D0301B5000130861803016F
:10089000350403194C2C0515851585140130A90064
:1008A000F430B9200511851185100130A9004A30B6
:1008B000B920C40A372B01204E3062206F306220ED
:1008C00020306220733062206930622067306220FD
:1008D0006E306220613062206C30622020308400F3
:1008E0006030B220A03084005030B220203084002C
:1008F0003030B1200618B616061CB61203010618D1
:10090000013EB61A013C031D8B2CB70A0319B80A25
:100910000130B8207E2C0301B61A0130013A0319C8
:10092000B612031DB61603010618013EB61A013CA5
:10093000031DA02CB70A0319B80A0130B820932C64
:1009400003303802DE300319370203186E2C3614D8
:02095000282A53
:02400E00503F21
:00000001FF
